:10000000031E080085015F30A000213084008001BC
:10001000840AA00B07282F2824208400073984068F
:100020000310840C840C840C041A841704128419A1
:10003000841684118A01820701340234043408349E
:10004000103420344034803407398A018207283440
:1000500029342A342B342C342D342E342F342830A8
:10006000A100A2012108362101300D213608A3008C
:10007000A001A401A501A601A701DD20D620A201AF
:100080002208362101300D213608A200220836212F
:1000900023082121031D3E282508A9002608AA00BF
:1000A0002708AB002D303921A5002C303921A600BE
:1000B0002B303921A7002908362125080D213608C3
:1000C000AD002D08362100302121031D80282A088B
:1000D000362126080D213608AD002D0836210030C6
:1000E0002121031D80282B08362127080D213608E1
:1000F000AD002D08362100302121031D8028B428B1
:100100002508362100302121031D9228260836219A
:1001100000302121031DAC28270836210030212181
:10012000031DAF282C303921362100302121031D39
:10013000A9282C303921362101302121031DB22874
:100140000830EF209630F6200830EB209630F6206D
:10015000A0280430A000B4280230A000B428013048
:10016000A000B428A001B4282008362100302121A5
:10017000031DD1282408362101300D213608A400A2
:100180002408362104302621031DC8280130A4008C
:100190002408362120082621031DCF28D128DD2060
:1001A00040280130B700F430F72040280230EB201F
:1001B0003230F6200230EF2041290030EF20643049
:1001C000F6200030EB200130B7009030F7204129B5
:1001D00007300421E8280C20FF3A8005F3280C2082
:1001E0008004F228FF3A841780054129B701B60040
:1001F0001B2164003708360403190800F730FF3E5E
:10020000031DFF281D21F9288316F83881050F39B1
:10021000810463000F3081044129B901B8003630F0
:100220008400380880073908840F00000318013E55
:10023000031C80074129B709B609B60A0319B70A92
:100240000800B901B8002B2102394129B901B800D1
:100250002B210639412939083702031D3329380873
:10026000360203190234031C04340134B701B6000A
:1002700041290D20BD000005841B3D0603190034F3
:08028000013483126400080040
:02400E00DC3F95
:00000001FF
